:020000020000FC
:1000000027C018951895189518951895189518954E
:1000100038C018951895189518951895E0E6FF279B
:10002000662758D1AD9A50FFFDCF5527AD984D307A
:1000300011F42BD1F7CF483011F45BD1F3CF4A3014
:1000400089F3683279F363954193842F24D0EACF02
:100050000FED0DBF002701BB0CEF02BB899A8898FA
:1000600008E90AB907E109B9002703B900E204BBAE
:100070000FEF07BB00E80FBF07D000E20CB904D0B8
:10008000CDCF4CB15395189513E22FEF2A95F1F788
:100090001A95D9F708958CB95D9BFECF08957727FF
:1000A000623068F1E0E6FF270191033721F4019106
:1000B000023609F471E0E0E6FF270191033621F4EE
:1000C0000191023609F472E0E0E6FF270191023760
:1000D00021F40191023609F474E0E0E6FF27019172
:1000E000023721F40191013609F473E0E0E6FF27BD
:1000F0000191053621F40191093609F475E008955E
:10010000C895002021F0802DC6DF3196F9CF0895E3
:10011000EEE3F3E0F5DFE0E6FF27019101910191C5
:100120000032A1F4643091F401910053063070F470
:1001300080E2B1DF802F805DAEDFECE4F3E0E0DF52
:10014000402E90D008B3052908BB03C0EEEAF3E0C7
:10015000D7DF0895EAE5F3E0D3DFE0E6FF2701917A
:10016000019101910032A9F4643099F40191005396
:10017000063078F480E28FDF802F805D8CDFEAE646
:10018000F3E0BEDF402E6ED008B35094052108BBCB
:1001900003C0EEEAF3E0B4DF0895ECE8F3E0B0DF8B
:1001A000E0E6FF27019101910191003259F5643099
:1001B00049F50191003331F10053053018F507B9C5
:1001C000005D802F68DF8DE366DF84E264DF06EE8A
:1001D00006B95ADF24B015B0012D0F70902F16D03C
:1001E000892F59DF022D007F0295902F0FD0892F84
:1001F00052DF022D0F70902F09D0892F4CDF80E243
:100200004ADF03C0EEEAF3E07BDF0895905D9A33A6
:1002100008F0995F0895ECE7F3E072DFE0E6FF276E
:100220000191019101910032C9F46430B9F4019156
:100230000053083098F4023088F0402E13D030B2CA
:100240003520005D802F27DF8DE325DF332019F077
:1002500081E321DF06C080E31EDF03C0EEEAF3E0A6
:100260004FDF0895A1E05A2E442019F0550C4A940E
:10027000FBCF0895ECE9F3E043DFE0E6FF270191CF
:10028000802F09DF6A95D9F708958DE004DF8AE0B1
:1002900002DF05DF772319F4E8E0F3E031DF7130A6
:1002A00009F436DF723009F455DF733009F475DF75
:1002B000743009F4B0DF753009F4DCDF6627E0E65E
:1002C000FF278DE0E8DE8AE0E6DE8DE0E4DE8AE00E
:1002D000E2DE089500E00EBBE199FECFE09A0DB397
:1002E000002331F0802FD7DE0EB303950EBBF4CF81
:1002F0000895662341F002916A9588E0CCDE80E2A1
:10030000CADE88E0C8DE089553594E54415820454E
:1003100052524F52202D20617661696C61626C658A
:1003200020636F6D6D616E64733A2073622C20637D
:10033000622C2072622C2072612C2065690053456A
:100340005420424954202D20426974002068617372
:10035000206265656E2073657400434C45415220F0
:10036000424954202D204269740020686173206244
:1003700065656E20636C6561726564005245414439
:1003800020424954202D20426974200052454144A6
:1003900020414443202D2041444300004543484F21
:1003A00020494E505554202D20004F4B0000207006
:1003B0006172616D65746572206E6F7420616C6C22
:1003C0006F776564206F7220706172616D6574650E
:1003D000722073796E74617820696E636F727265D2
:0403E0006374210021
:00000001FF
